:020000003529A0
:08000800CF00030E83128C00EF
:0E0010000A0E8D00040E8E008A110A12382985
:1000200003309707970C970C7F3097050000970BCC
:10003000162808000000000000000000000000007A
:10004000970B1A2808009708031D272808000D3071
:1000500000000000FF3E031D28280000970B272802
:1000600008009608031D35280800CC30FF3E031D0C
:1000700036280000960B35280800FA30960031200B
:10008000FA3096003120FA3096003120FA3096008E
:100090003120950B3D280800A301A601A7011708F0
:1000A000A400A501A3190800181C5C282408A607B1
:1000B0000318A70A2508A707980C0310A40DA50D7F
:1000C000A30A5228A301A401A601A701A501251A8C
:1000D00008000310A60DA70D9B0D9C0DA30DA40DEC
:1000E0001E082402031D76281D082302031C7F28F6
:1000F0001D08A3021E08031CA403A4022614A50ABB
:1001000067288312110897006F3098004C2026084A
:100110009B0027089C000A309D009E016220260853
:100120009F0027089000F4301F078F00013003184C
:10013000900A900797010F089B0010089C00901FE1
:10014000A7289B099C099B0A03199C0A970A6430FB
:100150009D009E01622026089400171CB128940976
:10016000940A14089700643098004C2026089900DF
:1001700027089A0019080F029F001A0A03181A0884
:100180001002A000A1011F089B0020089C00A01FD6
:10019000CF289B099C099B0A03199C0AA10A0A30D3
:1001A0009D009E01622026089200211CD9289209F8
:1001B000920A14089700643098004C202608990091
:1001C00027089A0019080F02A1001A0A03181A0832
:1001D0001002A200120897000A3098004C2026084E
:1001E0009B0027089C000A309D009E016220260883
:1001F0009F002708A0001F0821029300FE308316ED
:1002000005058500FE3083120505970001301704AF
:100210008500130897001020120897001A20140870
:1002200097002320FE30831605058500FE308312DB
:10023000050585000800C030831681008112011673
:10024000F0300105831295000530150483168100F6
:1002500083128B178B165A309100033095003D2086
:100260009101033095003D202B298A110A121B2988
:1002700083120B1D3D2981200B110E0E84000D0EE3
:0C0280008A000C0E8300CF0E4F0E090008
:00000001FF
